:020000040000FA
:06000000FE300F306A28FB
:08000800A000030EA100831209
:10001000C31D3B288B1C34288B1031181628B11CAB
:10002000342864300102031833281A2800001828E5
:1000300019281A281B281C281D281E281F2820289C
:1000400021283110B114A810031005190314AA0DAA
:10005000A90DA80DB00B342831152A08AF002908C6
:10006000AE002808AD00B11081010B11210E8300F4
:10007000A00E200E090005194328831601178312CC
:10008000B23081005E2883160113831203140B190A
:100090000310A80DA90DAA0DAB0DAC0DAC16FF30C9
:1000A0002C02031D5E28FA302B02031D5E28311539
:1000B0002A08AF002908AE002808AD008B100B11EC
:0A00C000210E8300A00E200E09009F
:0C00D400203084008001840A8030040287
:1000E000031C6C281230B0005A30C000C10001302F
:1000F000D400D500E400E500E300F100F000073093
:10010000D8008030D7001F30E6000717FA30FD0016
:100110000330EF0083160F308505203086050D3043
:1001200087058312850186018701103083168E00B2
:100130008312703083168F008312003003179900EA
:100140000313003003179A000313003097000030A8
:100150009F00003083169F008312003003179E001B
:100160000313003003179F000313C0308316810070
:1001700083123130900000309200003083169400DA
:10018000831200309400A63083169800831200304A
:1001900083169B00831290309800333083169900A9
:1001A0008312003083168C008312003083168D007A
:1001B000831210308B000D16E92481018E018F010E
:1001C0000B118B100B108C128C018D010D168B17DF
:1001D00003234123782123213119B623311A3D21EC
:1001E000591CE622591877228F080319EB288F0132
:1001F000B9227723F421CF218F21AF210629E71BD4
:10020000EB01EB0B0629E801E901EA01E7135918B4
:10021000EB28B1191829D60BEB28B11A0A30B11EF8
:10022000C830D600B11A1F297821CC0ACC194A143B
:10023000B111B11A0A30B11EC830D600EB287821AE
:10024000BE18E924EB286400C31DB113C31D0800C8
:10025000311808000B1D08000B11B11031141230B9
:10026000B000051D3829B117831601138312080049
:10027000B113831601178312080031124A10CC0102
:1002800021305B02031D4A295C08CE005D08CF00C7
:10029000661773295B085C065D02031D0800773052
:1002A0005B02031D57295C087406C400732966307D
:1002B0005B02031D5E295C08CB00732955305B028D
:1002C000031D65295C08F800732944305B02031D97
:1002D0006C295C08FA00732933305B02031D732913
:1002E0005C08FB007329B116B1110A30D600080072
:1002F000591459158B138316071283128B1707167F
:1003000008005910D9101930DE00B112B111C830EF
:10031000D6008B138316071683128B170800051857
:1003200096291930C00703189B2908000A30C0021B
:10033000031CA7290800FF30C000421464304102AA
:10034000031808004210C2144317C3140800C00168
:100350004210C213C21C0800C201431308008518D2
:10036000B6291930C1070318BB2908000A30C10299
:10037000031CC7290800FF30C1004214643040024A
:1003800003180800421042154317C3100800C101AA
:100390004210C213421D0800C20143130800E303C8
:1003A000031D080065186008E518610865196208F2
:1003B00099000330E3000310E50DE519E02908007A
:1003C0001430E3000130E5001030E61AE40020307C
:1003D000661BE4000310E40D03186414640866054A
:1003E0000319E029032308008C1E0800E7174A15AB
:1003F0000717FA30FD001819CA146908E8006A08DE
:10040000E9001A08EA00E81F08006808C13C031D5B
:10041000102A69086A05C3046A096904C305762AB3
:100420006808C23C031D1B2A69086A05C5046A09DD
:100430006904C505762A6808C43C031D222A690898
:10044000F700762A6808FC39E03C031D322A690867
:1004500068188038BB006A08E8188038BA00CD24D4
:10046000BE14762A6808FC39F03C031D4C2A690842
:1004700068188038EC0064000D1E3C2A8B136C0851
:1004800003178D0083168C130C1483120C080313AE
:10049000ED008B17E616762A6808FC39803C031DB0
:1004A0005B2A690868188038CE006A08E818803826
:1004B000CF00D815762A6808FC39903C031D662ABF
:1004C000690868188038CE005816762A6808A03C5B
:1004D000031D762A69086A188038CD00C310EA180F
:1004E000C31445126A194516D816762A08005919F8
:1004F000842AD3030F305305031D0800D3080319C2
:10050000872A0716D30E0800591B4D2359130712CB
:100510005911D918812955185008D518510855195D
:1005200052085705031D972AFF30D3009A2A22301C
:10053000D3009A2A0310D70C03189F2A0800803092
:10054000D7000310D50DD519A62A08000130D50013
:100550000430D819D4000830581AD4000310D40D30
:1005600003185414540858050319A62A4123D91412
:100570000800EF0B08000330EF00061EE42A051602
:100580000310F00D031CD22A0130F0000310F10D0E
:10059000711ED22A0130F100F0004408F300C31AA2
:1005A000F317051271187308F1187208711977089A
:1005B000F11DDD2A4B084A18803870050612031910
:1005C0008516031D8512080006160800DA0A0319AD
:1005D000D9165916071E5912D91DFF2A591AFF2A72
:1005E000B1155A08283CD91A0310DD0DDC0DDB0DBE
:1005F000DA01D912DE0BFF2A31161930DE00D915C7
:10060000591ED9110800E001E101E201641F0F2B1E
:100610004830E0004E08E1004F08E2006613E41E97
:10062000182B4730E0006C08E1006D08E200E6128C
:10063000641E202B4130E0007A08E1007B08E200D4
:10064000E41D282B4C30E0007708E1007808E20038
:10065000641D302B4530E0004A08E1004B08E20001
:10066000E41C382B4630E0004308E1004408E20077
:10067000641C402B5830E0005930E1005A30E20051
:100680000800D001D101D201541C4B2BF730D0000F
:100690004308D100732BD41C522BA130D000770813
:1006A000D100732B541D592BA230D0004508D10026
:1006B000732BD41D632BC130D0004E08D1004F08DE
:1006C000D200D8110800541E6B2BC230D0004E0847
:1006D000D1005812732BD41E0800A730D0004D084B
:1006E000D100D812732B50085106D2000800311FD8
:1006F0007C2BFC0303193113071F812BFD03031906
:100700000713031044180314B20DF030320203191A
:10071000431307184311071C43150719C311071D7D
:10072000C315751C972BC31E8710C31A8714FE0BA5
:10073000080044182B25441C87124A1C87174A18A6
:100740002325790AF71BF707771BAA2B790A77026B
:100750000318F7007808F2000310790C013E7802C4
:10076000C3120318F2000318C31608003111311B1D
:100770000800591808004A100717FA30FD00B701A1
:100780000430B8000C30370230300318B807C319F2
:10079000B8178B1320303707380703178D008316DF
:1007A0008C130C1483120C080313A400A500C03092
:1007B000A50610303707380703178D0083168C13F2
:1007C0000C1483120C080313A300A6000230A60623
:1007D00000303707380703178D0083168C130C146D
:1007E00083120C080313A200A7000130A7068B1781
:1007F000B11F002C22090339A200A309A409A509ED
:10080000C31D0F2C22082D02031D982C23082E0235
:10081000031D982C24082F02031D5C2C1B2C24087C
:100820002F02031D982C23082E02031D5C2C220886
:100830002D02031D982C00303702031D232C3D147C
:100840003E144314080001303702031D312CFA30E6
:10085000FC003117431FC314431FB0244030C306AC
:10086000080002303702031D3F2CFA30FC0031171C
:10087000431FC314431FB8244030C306080003308D
:100880003702031D462C431FC314080064000D1ECD
:10089000472C3030370738077F3903178D00831610
:1008A0008C130C1483120C080313F7005917FA3039
:1008B000FC0031174030C306C31D632C25082F02EE
:1008C000031D982C6B2C26082E02031D982C27083C
:1008D0002D02031D982C00303702031D752C3D1C82
:1008E000752C3D103E144310080001303702031DE3
:1008F000832CFA30FC003117431FC310431FA72479
:100900004030C306080002303702031D912CFA3034
:10091000FC003117431FC310431FB8244030C306E7
:10092000080003303702031D982C431FC310080032
:10093000B70A1C30370203180800C02B3E1C080001
:100940003E101030BB003D08BA00CD2408005917F6
:10095000C310780AF700790A77020318F700080035
:100960005917C3147803F700790AF71BF707080033
:1009700059170310790C78077902031CC72C031947
:10098000C72C0310790C013E7807F700080003100C
:10099000790C013E7802F70008000D123B08831223
:1009A00003178D00831203133A08831203178C0078
:1009B000831603178C130C158B138B1BDC2C5530F3
:1009C0008D00AA308D008C148B170C118312031329
:1009D000080064000D1EEA2CBE108B138B1BED2C3F
:1009E000313003178D0083168C130C1483120C08FE
:1009F0000313F4008B1774108B13323003178D0020
:100A000083168C130C1483120C080313F5008B1738
:100A10008B13333003178D0083168C130C14831241
:100A20000C080313F6008B178B13303003178D005F
:100A300083168C130C1483120C0803130718303020
:100A4000F900F90308000708803A87000800070842
:100A5000403A870008000708203A87000800070886
:060A6000023A87000800C5
:084000000F00000002000600A1
:02400E00CC03E1
:1042000000002600FF00FF0040004200440046007E
:104210004200430040004100460047004400450082
:10422000FF00FF00FF00FF00F200F600FA00FE00B2
:10423000F000F200F400F600F800FA00FC00FE00C6
:10424000FF00FF00FF00FF00E500E500E500E500DE
:10425000E900E900E900E900E900E900E900E90016
:104260001800000001000000FF00FF00FF00FF0039
:104270000000010002000300040005000600070022
:104280004300420041004000470046004500440012
:104290004400450046004700400041004200430002
:1042A000F000F200F400F600F800FA00FC00FE0056
:1042B000F000F200F400F600F800FA00FC00FE0046
:1042C000ED00ED00ED00ED00ED00ED00ED00ED0086
:1042D000F100F100F100F100F100F100F100F10056
:1042E000080009000A000B000C000D000E000F0072
:1042F0001000110012001300140015001600170022
:10430000FF00FF00FF00FF000000000000000000B1
:104310000300030003000300030003000300030085
:10432000FF00FF00FF00FF00C800C800C800C80071
:10433000C800C800C800C800C800C800C800C8003D
:10434000FF00FF00FF00FF00C300F300CF00FF00ED
:104350000300C3003300F3000F00CF003F00FF0055
:10436000FF00FF00FF00FF00FF00FF00FF00FF0055
:10437000FF00FF00FF00FF00FF00FF00FF00FF0045
:10438000020002000200020002000200020002001D
:10439000000000000000000000000000000000001D
:1043A000C800C800C800C800C800C800C800C800CD
:1043B00088008800880088008800880088008800BD
:1043C0000300C3003300F3000F00CF003F00FF00E5
:1043D0000300C3003300F3000F00CF003F00FF00D5
:1043E000FF00FF00FF00FF00FF00FF00FF00FF00D5
:1043F000FF00FF00FF00FF00FF00FF00FF00FF00C5
:00000001FF
